:100000000C942A000C945C101895000018950000C0
:10001000189500001895000018950000189500002C
:10002000189500001895000018950000189500001C
:10003000189500001895000018950000189500000C
:1000400018950000189500001895000018950000FC
:10005000189500008FE58DBFC0EDE8EC4E2E88E0CE
:100060008EBFD6E0F3E05F2EA89584B7082E877F79
:1000700084BF88E1992781BD91BDEEEFF7E0A0E64E
:10008000B0E088278D933197E9F780E189B980E066
:1000900080BD88E18AB96624D39AD29AD198B89A59
:1000A000B99ABA9ABB9ABC9AA298A39AA49AA59A0A
:1000B000A69AA79A8B9885B78C7F826085BFB59AE0
:1000C000B69A9A9AC99A839A78947BB770647BBFE0
:1000D00000EE1DE420EE30E0A6EBB0E00D931D93A2
:1000E0002D933C93A6EBB0E00D911D912D913C9189
:1000F000A2E0B1E00D931D932D933C93A2E0B1E0FB
:100100000D911D912D913C91A6E0B1E00D931D93B1
:100110002D933C93AAEFB0E0E8EEFFE20E9430138B
:1001200081E08093AB000091AB00023018F011F039
:100130000C94AC00DA9A84EF91E00E949911DA985D
:100140008AEF90E00E949911ABEAB0E08C918F5F4A
:100150008C9310F40C9493000E94060780E0809327
:100160000A0100910A01053018F011F00C94D0003A
:10017000ECE6F1E2AAE0B1E08C919927AAE0B1E0C7
:10018000AD90BB24A4ECB0E0AA0DBB1D0E944916A3
:10019000AAE0B1E08C918F5F8C9310F40C94B100C5
:1001A0005A924A92A6EBB0E00D911D912D913C918F
:1001B000D2010D931D932D933C9384E00E9417155B
:1001C0000E94270B229684E00E94BC105A924A9209
:1001D000A6EBB0E00D911D912D913C91D2010D93B4
:1001E0001D932D933C9384E00E9417150E94270BCA
:1001F000229684E00E94BC100E945701A6E0B1E064
:100200004D915D916D917C91A2E0B1E00D911D91B8
:100210002D913C910E94941611F40C9411010E94AE
:10022000EF03AAEBB0E04D915D916D917C91A6EB4F
:10023000B0E00D911D912D913C910E94941611F406
:100240000C9438015A924A92A6EBB0E00D911D91A0
:100250002D913C91D2010D931D932D933C9384E0FD
:100260000E9417150E94270B229684E00E94BC1062
:10027000A6EBB0E00D911D912D913C91AAEBB0E061
:100280000D931D932D933C93A9EAB0E04D915C91A1
:10029000A7EAB0E00D911C910417150711F40C9416
:1002A00053010E9426050E9491060C94E60081E00D
:1002B0000E94111581E00E94111582E00E94111523
:1002C00082E00E94111582E00E94111500E513ECF6
:1002D00020E030E0ADE3B1E00D931D932D933C930E
:1002E0000E949A17E4E2F0E30E942911A0E6B0E030
:1002F00036E20E94E3100E94971781E0E0E6F0E00A
:1003000002E00A93A0E9B0E00E943D17A0E6B0E049
:100310000E947D17EA2FFB2F32970FEFA3E9B0E081
:100320000E944417A0E9B0E0E8E2F0E30E948317DE
:1003300081E009F480E08F93A3E9B0E0ECE2F0E320
:100340000E94831781E009F480E09F91892B882324
:1003500011F40C94CD0181E0A885B9858C93A88512
:10036000B9850C91023018F011F00C94C901DA9A99
:1003700084E690E00E949911DA9884E690E00E9469
:100380009911A885B9858C918F5F8C9310F40C948A
:10039000AF010C9457010C94CE01DA9A85E0E0E6A7
:1003A000F0E009E00A93A7E8B0E00E943D17A7E853
:1003B000B0E00E940017A6EBB0E00D931D932D93C3
:1003C0003D93A6EBB0E00D911D912D913C91A8E1DC
:1003D000B1E00D931D932D933C9340E054E465E907
:1003E00078E0A6EBB0E00D911D912D913C910E941B
:1003F00094160CF402C00C941202A6EBB0E00D911E
:100400001D912D913C9144E050E060E070E00E942D
:100410001B15A6EBB0E00D931D932D933D93AC9867
:100420000C942502A6EBB0E00D911D912D913C910D
:1004300040E058E468EE71E00E948F16A6EBB0E051
:100440000D931D932D933D93AC9A82E1E0E6F0E08D
:1004500006E00A93A5E9B0E00E943D17A5E9B0E0E7
:100460000E940017A2EBB0E00D931D932D933D93D6
:10047000A2EBB0E00D911D912D913C9144E050E034
:1004800060E070E00E941B15A2EBB0E00D931D939D
:100490002D933D9386E0E0E6F0E003E00A93ACE9BB
:1004A000B0E00E943D17ACE9B0E00E940017A7EA57
:1004B000B0E00D931C938EE0E0E6F0E004E00A93D8
:1004C000A0EAB0E00E943D17A0EAB0E00E94001749
:1004D000AE81BF810C93AE81BF810C91003011F0D1
:1004E0000C947E0201E010E020E030E0A0E2B1E0F8
:1004F0000D931D932D933C930C943C03013011F00C
:100500000C948E020AE010E020E030E0A0E2B1E0BE
:100510000D931D932D933C930C943C030A3011F0E2
:100520000C949E0204E610E020E030E0A0E2B1E08E
:100530000D931D932D933C930C943C030B3011F0C1
:100540000C94AE0208EE13E020E030E0A0E2B1E04F
:100550000D931D932D933C930C943C030C3411F09C
:100560000C94BE0208E213E220E030E0A0E2B1E029
:100570000D931D932D933C930C943C03043611F082
:100580000C94CE0200E117E220E030E0A0E2B1E0FE
:100590000D931D932D933C930C943C03053611F061
:1005A0000C94DE0200EA16E821E030E0A0E2B1E0BF
:1005B0000D931D932D933C930C943C030E3611F038
:1005C0000C94EE0200E412E42FE030E0A0E2B1E08F
:1005D0000D931D932D933C930C943C030F3611F017
:1005E0000C94FE0200E816E928E930E0A0E2B1E050
:1005F0000D931D932D933C930C943C03083E11F0F6
:100600000C940E0302E310E020E030E0A0E2B1E041
:100610000D931D932D933C930C943C03093E11F0D4
:100620000C941E030AEF10E020E030E0A0E2B1E0FD
:100630000D931D932D933C930C943C03023F11F0BA
:100640000C942E0304EF11E020E030E0A0E2B1E0D2
:100650000D931D932D933C930C943C03033F11F099
:100660000C943C0308E813E120E030E0A0E2B1E0A4
:100670000D931D932D933C9388E1E0E6F0E001E0BB
:100680000A93AB81BC810E943D17AA81BB810E9465
:100690000017AFEAB0E00C9389E1E0E6F0E001E09A
:1006A0000A93A981BA810E943D17A881B9810E944D
:1006B0000017A0EBB0E00C938DE1E0E6F0E001E084
:1006C0000A93AD81BE810E943D17AC81BD810E941D
:1006D0000017AEEAB0E00C938EE1E0E6F0E001E056
:1006E0000A93A5EAB0E00E943D17A5EAB0E00E9497
:1006F0000017ADEAB0E00C93A3E3B0E00C9102FB6D
:1007000081E00EF080E08F930091AC00013081E039
:1007100009F480E09F918923882311F40C94A003AD
:1007200082E50E94301188E50E9430118BE30E941F
:100730003011DB98C49881E08093AC000C94C20324
:10074000A3E3B0E00C9102FB81E00EF480E08F9314
:100750000091AC00013081E009F080E09F91892395
:10076000882311F40C94C20384E50E94301188E5BB
:100770000E9430118BE30E943011DB9AC49A80E012
:100780008093AC000091AE00013011F00C94CC03CA
:10079000DB9AC49A0C94CE03DB98C4980091AD0008
:1007A000053081E009F080E08F930091AD000430C6
:1007B00081E009F080E09F91892B882311F40C944B
:1007C000E60381E08093B1000C94E90380E080931C
:1007D000B10088E0481A80E0580A2A960895A2E0FD
:1007E000B1E00D911D912D913C91A6E0B1E04D91AC
:1007F0005D916D917C910E948F16A4E1B1E00D9303
:100800001D932D933D93A4E1B1E00D911D912D9188
:100810003C9144E050E060E070E00E941B15A4E1D0
:10082000B1E00D931D932D933D93A4E1B1E00D91A3
:100830001D912D913C91A0E2B1E04D915D916D91A2
:100840007C910E941B15A4E1B1E00D931D932D93A3
:100850003D93AC9B0C943E04A4E1B1E00D911D913D
:100860002D913C9144E050E060E070E00E9437112F
:10087000A4E1B1E04D935D936D937D93A6EBB0E061
:100880000D911D912D913C91A4E1B1E04D915D91AF
:100890006D917C910E948A16A6EBB0E00D931D939A
:1008A0002D933D9340E452E46FE070E0A6EBB0E09E
:1008B0000D911D912D913C910E9494160CF402C053
:1008C0000C946C0400E412E42FE030E0A6EBB0E0FE
:1008D0000D931D932D933C9340E856E36EEB76E227
:1008E000A6EBB0E00D911D912D913C910E949416C4
:1008F0001CF011F00C947E040C94880400E815E5BB
:1009000028EC30E2A6EBB0E00D931D932D933C93C1
:10091000A2E0B1E00D911D912D913C91A6E0B1E0D6
:100920000D931D932D933C935A924A92A6EBB0E0FF
:100930000D911D912D913C91D2010D931D932D93FD
:100940003C9384E00E9417150E94270B229684E0B6
:100950000E94BC105A924A92A6EBB0E00D911D91F4
:100960002D913C91D2010D931D932D933C9384E0E6
:100970000E9417150E94C104229684E00E94BC10B8
:1009800008958CE00E9411158EE00E941115AC9B19
:100990000C94DE04AC81BD810D911D912D913C9193
:1009A00040E058E468EE71E00E948A16AC81BD8197
:1009B0000D931D932D933D930C94F004AC81BD8158
:1009C0000D911D912D913C9144E050E060E070E06C
:1009D0000E943711AC81BD814D935D936D937D93E2
:1009E000AA81BB81EC81FD810E94AA16EA81FB816C
:1009F000A0EBB3E00E943217E0EBF3E0AA81BB81E9
:100A0000112722270BE033270E944C16A881B981B9
:100A1000EEE2F0E30E943E15EA81FB81A881B981F4
:100A20000E94DA100E943217A881B9810E94DA1060
:100A3000ECE2F0E30E943E15A881B9810E942311E7
:100A40008AE1481A80E0580A24960895A7EAB0E09F
:100A50000D911C910A3050E015070CF402C00C9463
:100A600035050C9426050C948806A7EAB0E00D9194
:100A70001C91063252E015071CF011F00C9442054F
:100A80000C9446050C9426050C948806A7EAB0E061
:100A90000D911C910A3050E0150780E00CF081E0C8
:100AA0008F93A7EAB0E00D911C910E3150E015072D
:100AB00081E014F009F080E09F918923882311F4EC
:100AC0000C94660576E078BB0C948806A7EAB0E043
:100AD0000D911C910E3150E0150780E00CF081E083
:100AE0008F93A7EAB0E00D911C91023350E01507F7
:100AF00081E014F009F080E09F918923882311F4AC
:100B00000C94860575E078BB0C948806A7EAB0E0E3
:100B10000D911C91023350E0150780E00CF081E04C
:100B20008F93A7EAB0E00D911C91003550E01507B6
:100B300081E014F009F080E09F918923882311F46B
:100B40000C94A60574E078BB0C948806A7EAB0E084
:100B50000D911C91003550E0150780E00CF081E00C
:100B60008F93A7EAB0E00D911C91083750E015076C
:100B700081E014F009F080E09F918923882311F42B
:100B80000C94C60573E078BB0C948806A7EAB0E025
:100B90000D911C91083750E0150780E00CF081E0C2
:100BA0008F93A7EAB0E00D911C91003A50E0150731
:100BB00081E014F009F080E09F918923882311F4EB
:100BC0000C94E60572E078BB0C948806A7EAB0E0C6
:100BD0000D911C91003A50E0150780E00CF081E087
:100BE0008F93A7EAB0E00D911C910E3B50E01507E2
:100BF00081E014F009F080E09F918923882311F4AB
:100C00000C94060671E078BB0C948806A7EAB0E065
:100C10000D911C910E3B50E0150780E00CF081E037
:100C20008F93A7EAB0E00D911C910C3D50E01507A1
:100C300081E014F009F080E09F918923882311F46A
:100C40000C94260670E078BB0C948806A7EAB0E006
:100C50000D911C910C3D50E0150780E00CF081E0F7
:100C60008F93A7EAB0E00D911C910E3051E015076B
:100C700081E014F009F080E09F918923882311F42A
:100C80000C94460679E078BB0C948806A7EAB0E09D
:100C90000D911C910E3051E0150780E00CF081E0C1
:100CA0008F93A7EAB0E00D911C91003951E0150730
:100CB00081E014F009F080E09F918923882311F4EA
:100CC0000C94660678E078BB0C948806A7EAB0E03E
:100CD0000D911C91003951E0150780E00CF081E086
:100CE0008F93A7EAB0E00D911C91063252E01507F0
:100CF00081E014F009F080E09F918923882311F4AA
:100D00000C94860677E078BB0C9488060C94260534
:100D1000A7EAB0E08D919C91A9EAB0E08D939C93F5
:100D2000089587E00E94111585E00E94111581E069
:100D30000E941115A4E2B1E08C918F5F8C93009119
:100D40002401043111F00C94FE0680E0809324010C
:100D50000E949A17E2E3F0E30E942911AC81BD8161
:100D600036E00E94E3100E94971781E0EC81FD813C
:100D700004E00A93AB81BC810E943D17AA81BB812C
:100D8000E8E3F0E30E94831711F40C94CB060C9473
:100D900000070C94DB0685E0EC81FD8101E00A93FD
:100DA000AB81BC810E943D17AA81BB810E940017C4
:100DB000A881B9810C93A881B9810C91013011F0FF
:100DC0000C94E506AF9A0C94E606AF98A881B98119
:100DD0000C91023011F00C94F006AE9A0C94F106CE
:100DE000AE98A881B9810C91033011F00C94FB06E8
:100DF000AD9A0C94FC06AD980C9400070C94000777
:100E00008DE0481A80E0580A2696089581E00E94F5
:100E1000111581E00E94111584E00E941115AC812A
:100E2000BD81BA93AA935A924A9287E8D2018C93D1
:100E300081E00E9417150E943D10249681E00E94D7
:100E4000BC10AC81BD818C9181608C935A924A9286
:100E500087E8D2018C9381E00E9417155A924A923A
:100E6000A885B9858C91D2018C9381E00E941715D9
:100E70000E942B10249682E00E94BC1081E0AC817D
:100E8000BD818C93AC81BD810C91003011F40C9428
:100E90006207AC81BD81BA93AA935A924A9287E8BD
:100EA000D2018C9381E00E9417150E943D10249678
:100EB00081E00E94BC10AC81BD818C9181708C93CB
:100EC0000C94420781E080930A0100910A010630E8
:100ED00018F011F00C94940700910A0146E0040FF9
:100EE000ABE0B1E00C93AAE0B1E0AD90BB24ADEB78
:100EF000B0E0AA0DBB1DBA93AA935A924A92809170
:100F00000B01D2018C9381E00E9417150E943D10C5
:100F1000249681E00E94BC10AAE0B1E08C918F5F22
:100F20008C9310F40C946507AEEBB0E00C91112794
:100F30002227332740EE50E060E070E00E948B11E2
:100F4000AAECB0E00D931D932D933D9395E0AAEC90
:100F5000B0E00E946515AAECB0E00D911D912D91B5
:100F60003C9144E050E060E070E00E948A16AAECF8
:100F7000B0E00D931D932D933D930091BE004FE182
:100F80000423AC81BD810C9392E0AC81BD810E94B1
:100F900044150091BF0040EC0423AA81BB810C934F
:100FA00096E0AA81BB810E945D15AC81BD810C9148
:100FB000112722273327AA81BB814C915527662709
:100FC00077270E948A16AEECB0E00D931D932D9307
:100FD0003D9340E050E060E070E0AEECB0E00D9199
:100FE0001D912D913C910E94941611F00C940408CF
:100FF00001E010E020E030E0AEECB0E00D931D9396
:101000002D933C930C9424080091CE0041E00423DE
:10101000AC81BD810C93AC81BD810C91003011F489
:101020000C942408AEECB0E00D911D912D913C91F3
:1010300041E050E060E070E00E948A16AEECB0E063
:101040000D931D932D933D93AFEBB0E00C911127C1
:10105000222733274FE350E060E070E00E948B11BD
:10106000A881B9810D931D932D933D9394E0A881A0
:10107000B9810E944C150091C00040EF0423AC815F
:10108000BD810C9394E0AC81BD810E945D15A88167
:10109000B9810D911D912D913C91AC81BD814C91F7
:1010A0005527662777270E948A16A881B9810D9354
:1010B0001D932D933D93A881B981ECE0F1E00E944E
:1010C0007A14A0ECB0E00C911127222733274FE0CF
:1010D00050E060E070E00E948B11A881B9810D930F
:1010E0001D932D933D9398E0A881B9810E944C15E2
:1010F000A881B9810D911D912D913C91A1ECB0E099
:101100004C915527662777270E948A16A881B981B6
:101110000D931D932D933D9398E0A881B9810E9472
:101120004C15A881B9810D911D912D913C91A2EC96
:10113000B0E04C915527662777270E948A16A88130
:10114000B9810D931D932D933D9398E0A881B981AA
:101150000E944C15A881B9810D911D912D913C9152
:10116000A3ECB0E04C915527662777270E948A169A
:10117000A881B9810D931D932D933D93A881B981C9
:10118000EAEDF0E00E947A14AAEDB0E0BA93AA93D7
:10119000E0EFFFE2A2EDB0E00E943013EAEDF0E0F4
:1011A0000E9467122296AAEDB0E0BA93AA93AAED24
:1011B000B0E0ECE0F1E00E94C0112296AAECB0E0B1
:1011C000ECE0F1E00E947A14A2EEB0E0BA93AA93A8
:1011D000E8EFFFE2A2EDB0E00E943013E2EDF0E0B4
:1011E000ACE0B1E00E94FB112296AEECB0E0ECE086
:1011F000F1E00E947A14A2EEB0E0BA93AA93ACE0B8
:10120000B1E0E2EEF0E00E94FB112296A2EEB0E027
:10121000BA93AA93AAEDB0E0E2EEF0E00E94671262
:101220002296E2EEF0E0AAEEB0E00E944F13A2EFA9
:10123000B0E0E0E0F0E098E00E946617A2EFB0E0D6
:10124000E0E0F0E30E94091380E010F009F081E093
:101250008F93A2EFB0E0E8E0F0E30E94091381E091
:1012600008F080E09F91892B882311F40C944009A9
:10127000A2EEB0E0E0E1F0E30E9430130C944609E6
:10128000E2EFF0E0A2EEB0E00E944F1386E0481AD1
:1012900080E0580A2696089584E00E94111584E0A3
:1012A0000E94111584E00E94111584E00E9411151E
:1012B0009AE0A885B9850E94651505E51DE724E536
:1012C00030E0A885B9854D915D916D917C910E942A
:1012D0003711AC81BD814D935D936D937D9308E48F
:1012E00015E428E430E0A885B9854D915D916D91B4
:1012F0007C910E943711AE81BF814D935D936D93B8
:101300007D9392E0AC81BD810E946515AC81BD8169
:101310000C9142E00E946D17ABE0B1E08C9300911C
:101320000B01013011F00C94A709AC81BD810D9126
:101330001D912D913C9141E050E060E070E00E94F1
:101340008A16AC81BD810D931D932D933D93AE8183
:10135000BF810D911D912D913C914BE050E060E0DB
:1013600070E00E943711AE81BF814D935D936D9304
:101370007D93AE81BF810C9142E00E946D17ABE07E
:10138000B1E08C9300910B01013011F00C94DA095B
:10139000AE81BF810D911D912D913C9141E050E0B6
:1013A00060E070E00E948F16AE81BF810D931D93A7
:1013B0002D933D93AE81BF810D911D912D913C9157
:1013C00041E050E060E070E00E948A16AE81BF818B
:1013D0000D931D932D933D9340E850E060E070E045
:1013E000AC81BD810D911D912D913C910E9494166F
:1013F0001CF011F00C94FE090C94080A00E810E0AF
:1014000020E030E0AC81BD810D931D932D933C9382
:1014100040E050E060E070E0AE81BF810D911D9131
:101420002D913C910E9494161CF011F00C94220A0C
:1014300001E010E020E030E0AE81BF810D931D930C
:101440002D933C9300E010E020E030E0A881B981CA
:101450000D931D932D933C9381E080930A0100919D
:101460000A01063018F011F00C94FD0AA885B98520
:101470000D911D912D913C91AAE0B1E0AD90BB245E
:10148000A3ECB0E0AA0DBB1D4C915527662777272A
:101490000E941B15AA81BB810D931D932D933D9333
:1014A000AA81BB810D911D912D913C91AC81BD8193
:1014B0004D915D916D917C910E941B15AA81BB811C
:1014C0000D931D932D933D9348E455E468E470E03B
:1014D000AA81BB810D911D912D913C910E94941682
:1014E0000CF002C00C94F50A45E55DE764E570E098
:1014F000AA81BB810D911D912D913C910E94941662
:101500001CF011F00C94F50A40E050E060E070E04F
:10151000A881B9810D911D912D913C910E94941645
:1015200011F00C94BB0AAA81BB810D911D912D91E4
:101530003C91A881B9810D931D932D933C93AAE012
:10154000B1E0AD90BB24A3ECB0E0AA0DBB1D8C9123
:10155000AAECB0E08D9388278D938D938C93AC810A
:10156000BD810D911D912D913C91AEECB0E00D939C
:101570001D932D933C93A881B9814D915D916D91FF
:101580007C91AA81BB810D911D912D913C910E946E
:1015900094161CF011F00C94F50AAA81BB810D91F0
:1015A0001D912D913C91A881B9810D931D932D938F
:1015B0003C93AAE0B1E0AD90BB24A3ECB0E0AA0D4F
:1015C000BB1D8C91AAECB0E08D9388278D938D93F1
:1015D0008C93AC81BD810D911D912D913C91AEEC10
:1015E000B0E00D931D932D933C93AAE0B1E08C9154
:1015F0008F5F8C9310F40C942F0AAC81BD810D91F8
:101600001D912D913C9142E050E060E070E00E941D
:101610008F16AC81BD810D931D932D933D93AE81AB
:10162000BF814D915D916D917C91AC81BD810D919A
:101630001D912D913C910E9494161CF011F00C9478
:101640002C0A80E1481A80E0580A2896089584E020
:101650000E94111584E00E94111584E00E9411156A
:1016600081E00E94111581E00E94111581E00E9425
:10167000111581E00E94111581E00E94111588E08A
:101680000E94111584E00E94111584E00E9411153A
:101690000091AE00003081E009F080E08F9300916E
:1016A000AF00003081E009F080E09F9189238F93A3
:1016B0000091B000003081E009F080E09F91892323
:1016C000882311F40C94760BA6EBB0E00D911D91DC
:1016D0002D913C9140EA5CE860E070E00E948F163A
:1016E000AE89BF890D931D932D933D930091AE005C
:1016F000003081E009F080E08F930091AF0000306E
:1017000081E009F080E09F9189238F930091B000E0
:10171000013081E009F080E09F918923882311F452
:101720000C94A40BA6EBB0E00D911D912D913C9172
:1017300040EA5CE860E070E00E948F16AE89BF89E5
:101740000D931D932D933D930091AE00003081E0E9
:1017500009F080E08F930091AF00013081E009F043
:1017600080E09F9189238F930091B000013081E048
:1017700009F080E09F918923882311F40C94E60BF3
:10178000A6EBB0E00D911D912D913C9140EA5CE8F3
:1017900060E070E00E948F16AE89BF890D931D93A3
:1017A0002D933D93AE89BF890D911D912D913C9153
:1017B000A2EBB0E04D915D916D917C910E948A16F3
:1017C000AE89BF890D931D932D933D930091AE007B
:1017D000003081E009F080E08F930091AF0001308C
:1017E00081E009F080E09F9189238F930091B00000
:1017F000003081E009F080E09F918923882311F473
:101800000C94280CA6EBB0E00D911D912D913C910C
:1018100040EA5CE860E070E00E948F16AE89BF8904
:101820000D931D932D933D93AE89BF890D911D910D
:101830002D913C91A2EBB0E04D915D916D917C9129
:101840000E948A16AE89BF890D931D932D933D93F7
:101850000091AE00013081E009F080E08F930091AB
:10186000AF00003081E009F080E09F9189238F93E1
:101870000091B000003081E009F080E09F91892361
:10188000882311F40C94500CA6EBB0E00D911D913F
:101890002D913C91AE89BF890D931D932D933C935F
:1018A0000091AE00013081E009F080E08F9300915B
:1018B000AF00013081E009F080E09F9189238F9390
:1018C0000091B000003081E009F080E09F91892311
:1018D000882311F40C94780CA6EBB0E00D911D91C7
:1018E0002D913C91AE89BF890D931D932D933C930F
:1018F0000091AE00013081E009F080E08F9300910B
:10190000AF00013081E009F080E09F9189238F933F
:101910000091B000013081E009F080E09F918923BF
:10192000882311F40C94A80CA6EBB0E00D911D9146
:101930002D913C91A2EBB0E04D915D916D917C9128
:101940000E948A16AE89BF890D931D932D933D93F6
:101950000091AE00013081E009F080E08F930091AA
:10196000AF00003081E009F080E09F9189238F93E0
:101970000091B000013081E009F080E09F9189235F
:10198000882311F40C94D80CA6EBB0E00D911D91B6
:101990002D913C91A2EBB0E04D915D916D917C91C8
:1019A0000E948A16AE89BF890D931D932D933D9396
:1019B0000091B100013081E009F080E08F93009147
:1019C000AE00013081E009F080E09F9189238823F7
:1019D00011F40C94FD0CAE89BF890D911D912D91D0
:1019E0003C9140EE5BEA60E070E00E948F16AE89A9
:1019F000BF890D931D932D933D935A924A92A88DC2
:101A0000B98D0D911D912D913C91D2010D931D9396
:101A10002D933C9384E00E9417150E944C09229656
:101A200084E00E94BC10AAECB0E0ECE0F1E00E947F
:101A30007A14AE89BF89EC81FD810E947A14AAEDE7
:101A4000B0E0BA93AA93AE81BF81ECE0F1E00E94CE
:101A5000FB112296AEECB0E0ECE0F1E00E947A14CB
:101A6000AAEDB0E0BA93AA93ACE0B1E0EAEDF0E001
:101A70000E94FB112296C9990C94660DAAEFB0E062
:101A8000BA93AA93E8E1F0E3A2EDB0E00E9430132C
:101A9000EAEFF0E00E94FB112296A2EEB0E0BA93CA
:101AA000AA93AAEFB0E0E2EEF0E00E94C011229605
:101AB000AAEFB0E0E8EEFFE20E943013E0E0F0E0D1
:101AC000A2EEB0E098E07BE70E945517AAEDB0E0E7
:101AD000BA93AA93A2EEB0E0EAEDF0E00E9467129A
:101AE000229681E080930A0100910A01063018F0E5
:101AF00011F00C948D0D80E0AAE0B1E0AD90BB2414
:101B0000ADEBB0E0AA0DBB1D8C93AAE0B1E08C91C7
:101B10008F5F8C9310F40C94740DAAECB0E00D91CF
:101B20001D912D913C9144E050E060E070E00E94F6
:101B30008F16AAECB0E00D931D932D933D9395E085
:101B4000AAECB0E00E944C158091CA008093BE00C0
:101B500041E050E060E070E0AEECB0E00D911D912E
:101B60002D913C910E94941611F00C94C30D00E04D
:101B700010E020E030E0AEECB0E00D931D932D932B
:101B80003C930C94E30D0091CE0041E00423AC851E
:101B9000BD850C93AC85BD850C91003011F00C9483
:101BA000E30DAEECB0E00D911D912D913C9141E023
:101BB00050E060E070E00E948F16AEECB0E00D9354
:101BC0001D932D933D930091BE0040EE0423AA8502
:101BD000BB850C938091CE00A885B9858C9392E04B
:101BE000A885B9850E945D15AA85BB850C91A8853D
:101BF000B9854C91042BAEEBB0E00C930091CE0074
:101C000043E00423AE81BF810C9396E0AE81BF8197
:101C10000E944415AE81BF818C918093BF00EAED94
:101C2000F0E0ACE0B1E00E94B212AC81BD81BA93A9
:101C3000AA93ACE0B1E0EAEDF0E00E94AB1122968D
:101C4000EC81FD81AA81BB810E94981494E0AA8155
:101C5000BB810E946515AA81BB810C914FE30423CF
:101C6000AE85BF850C930091BF00AE85BF854C91BA
:101C7000042BAFEBB0E00C93ACE0B1E0BA93AA93C5
:101C8000E0EFFFE2A2EDB0E00E943013ECE0F1E003
:101C90000E94FB112296ECE0F1E0A881B9810E943C
:101CA0009814A881B9810D911D912D913C91AC8919
:101CB000BD890D931D932D933C9398E1AC89BD890B
:101CC0000E946515AC89BD890C914FEF0423A0ECEF
:101CD000B0E00C93EC81FD81AA81BB810E94981435
:101CE00094E0AA81BB810E944C150091C000AA819A
:101CF000BB814C91042BA0ECB0E00C93A881B9817E
:101D00000D911D912D913C91AA89BB890D931D9335
:101D10002D933C9390E1AA89BB890E946515AA89FD
:101D2000BB890C914FEF0423A1ECB0E00C93A88188
:101D3000B9810D911D912D913C91A889B9890D937F
:101D40001D932D933C9398E0A889B9890E9465154D
:101D5000A889B9890C914FEF0423A2ECB0E00C9351
:101D6000A881B9810C914FEF0423A3ECB0E00C9350
:101D7000AE85BF85BA93AA935A924A9289E8D20156
:101D80008C9381E00E9417150E943D10249681E0FB
:101D90000E94BC10AE85BF858C9180618C935A9255
:101DA0004A9289E8D2018C9381E00E9417155A92D9
:101DB0004A92AA89BB898C91D2018C9381E00E94BE
:101DC00017150E942B10249682E00E94BC1081E01F
:101DD00080930A0100910A01063018F011F00C946A
:101DE0001F0F00910A0146E0040FABE0B1E00C9335
:101DF0005A924A9280910B01D2018C9381E00E9409
:101E000017155A924A92AAE0B1E0AD90BB24ADEB0F
:101E1000B0E0AA0DBB1D8C91D2018C9381E00E9491
:101E200017150E942B10249682E00E94BC10AAE095
:101E3000B1E08C918F5F8C9310F40C94EA0EAE8518
:101E4000BF85BA93AA935A924A9289E8D2018C9399
:101E500081E00E9417150E943D10249681E00E94A7
:101E6000BC10AE85BF858C918F7E8C935A924A921E
:101E700089E8D2018C9381E00E9417155A924A9208
:101E8000AA89BB898C91D2018C9381E00E9417159D
:101E90000E942B10249682E00E94BC10AE85BF8564
:101EA000BA93AA935A924A9287E8D2018C9381E01E
:101EB0000E9417150E943D10249681E00E94BC10DC
:101EC000AE85BF858C9180648C93A9E2B1E04D9181
:101ED0005D916D917C91A8E1B1E00D911D912D91E5
:101EE0003C910E94941680E00CF081E08F93ADE26B
:101EF000B1E04D915D916D917C91A8E1B1E00D91C2
:101F00001D912D913C910E94941681E014F009F0EE
:101F100080E09F91892B882311F40C942510A8E16F
:101F2000B1E00D911D912D913C91A5E2B1E00D9391
:101F30001D932D933C93E8E1F1E00E94AA150E94C5
:101F4000C915A1E3B1E00E94ED15E0E2F0E30E94C3
:101F50003416E1E3F1E00E94AA150E94FF15EDE0BE
:101F6000F0E0A1E3B1E00E943717E1E3F1E00E9465
:101F70007615A5E3B1E0EDE0FF270E943717A5E253
:101F8000B1E00D911D912D913C91A5E3B1E04D91F2
:101F90005D916D917C910E948A16A9E2B1E00D934A
:101FA0001D932D933D93A5E2B1E00D911D912D91CF
:101FB0003C91A5E3B1E04D915D916D917C910E94C2
:101FC0008F16ADE2B1E00D931D932D933D935A9280
:101FD0004A9287E8D2018C9381E00E9417155A92A9
:101FE0004A92AA89BB898C91D2018C9381E00E948C
:101FF00017150E942B10249682E00E94BC1081E0ED
:10200000AE85BF858C93AE85BF850C91003011F4F1
:102010000C942310AE85BF85BA93AA935A924A9224
:1020200087E8D2018C9381E00E9417150E943D1031
:10203000249681E00E94BC10AE85BF858C9180748F
:102040008C930C9403100C94251081E2481A80E0C4
:10205000580A669608950E94A2171AEA0E94BA17B3
:10206000AA81BB811C910E94BA17A881B9811C91D9
:102070000E94BA170E94B117089580E08093410131
:102080000E94A2171AEA0E94BA17A881B9811C916E
:102090000E94BA170E94A2171BEA0E94BA170E9458
:1020A000D717A1E4B1E01C930E94B11780914101C0
:1020B000AA81BB818C9308950F921F922F923F9219
:1020C0004F925F927F92AF92BF920F931F932F9385
:1020D0003F934F935F936F937F938F939F93AF93B0
:1020E000BF93CF93DF93EF93FF938FB78F93C99BEA
:1020F0000C94891083990C948310A2E0B1E00E94A3
:10210000C0100C948710A2E0B1E00E94CD100C9496
:10211000981083990C949410AAEFB0E0AAEFB0E065
:102120000E94E7120C949810AAEFB0E00E94EA1205
:1021300070E47ABF8F918FBFFF91EF91DF91CF91C4
:10214000BF91AF919F918F917F916F915F914F91CF
:102150003F912F911F910F91BF90AF907F905F9013
:102160004F903F902F901F900F90189504050607F1
:10217000090B481A590A0895481A8827580A0895D9
:102180000D911D912D913C910F5F1F4F2F4F3F4F90
:102190003C932E931E930E9308950D911D912D91B6
:1021A0003C9101501040204030403C932E931E93B0
:1021B0000E9308958F938D918823E9F711978F914E
:1021C0000895A0EBB3E01AD0803089F0883091F008
:1021D0008D3039F03323B9F38D933A9563FE40D0B7
:1021E000F2CF63FC04C08DE03BD08AE039D0882771
:1021F0008C93089535D011973395E5CF0F931F93A6
:102200002F933F93AF93BF93ADE3B1E00D911D9139
:102210002D913C915F990BC08827802B812B822BBD
:10222000832B39F00150104020403040F3CF8CB167
:1022300001C08827BF91AF913F912F911F910F91BE
:102240000895A0EBB3E08D91882311F009D0FBCF66
:1022500008950E943016802D11F002D0FACF089513
:102260005D9BFECF8CB9089500FC05D0089530D059
:1022700005D001F8F9CF37D03FD00895842F952F9E
:10228000A62FB72FE894452B462B472B11F46894C3
:102290000895402F512F622F732F002711272227D7
:1022A0003327F0E2440F551F661F771F001F111FD1
:1022B000221F331F081B190B2A0B3B0B416028F40C
:1022C000080F191F2A1F3B1F4E7FFA9559F70895D3
:1022D0000024E89477FF02C006D0689400F809D083
:1022E00010F80124089512D04F5F5F4F6F4F7F4F5A
:1022F0000895E89437FF089500951095209530953E
:102300000F5F1F4F2F4F3F4F689408954095509592
:102310006095709508950423152326233723089587
:102320003197F1F70895689462F80895E89462F897
:102330000895EF93FF93EE27E82BE92B31F0E0EAC5
:10234000FFE03197F1F70197D1F7FF91EF910895F1
:102350007CD204D09EC10F0101D09EC1FD01FF932C
:10236000EF9387818F9390E889278783F0010BD0C3
:102370008F91EF91FF918783089567D204D089C12F
:102380000F0101D089C100E077D209F008959A01C8
:10239000281B390B1AF4D0010F01F5CF0027273382
:1023A000300708F09CC2822FA7D1BBD1C9D1372FEB
:1023B00036270AF4EDD1F0018081A80E8181B81E84
:1023C0008281C81E8381D81E8481E81E8581F81E03
:1023D00086818F708061081F1AF4DAD180E868273F
:1023E00005FF02C081E0AAD104FD01C004D2C2C130
:1023F0002CD204D04EC10F0101D04EC108E13CD215
:1024000009F00895480F591F4F5F534067276F9396
:102410005F934F9320D22227F00179D193E0110FDF
:10242000331F441F551F661F771F881F9A95B9F7E2
:10243000FD01A7E0BB279191A13011F49F7090613D
:10244000992301F1939FA00CB11CBB1F959FB695DA
:10245000C01CD11CBB1F979FB695E01CF11C0B1F25
:10246000919F200DA11CBB1F949FB695B01CC11C51
:10247000BB1F969FB695D01CE11CBB1F989FB695BD
:10248000F01C011DAA9549F02A2DAB2CBC2CCD2C9B
:10249000DE2CEF2CF02E0027CECF4F915F916F9165
:1024A00004FB16F05ED102C04F5F5F4F63C1FF9324
:1024B00009901124F8E0069408F4190E1794079473
:1024C000FA95D1F7FF910895C0D104D0E2C00F0171
:1024D00001D0E2C004E2D0D109F00895481B590BA5
:1024E00041505C4F67276F935F934F93F00104D186
:1024F0002FEFFD010CD1ADE3BA2FB77019F4209581
:102500002F932FEFA116B306C406D506E606F706ED
:10251000080738F0A11AB30AC40AD50AE60AF70A6E
:10252000080B221FAA0CBB1CCC1CDD1CEE1CFF1CC4
:10253000001FAA9509F72095AF90BF90CF90DF902C
:10254000EF90FF900F914F915F916F9104FB1EF000
:1025500008D1415050400EC1E881F981AA81BB8168
:102560000895FADF02D0FD0182C0A1D0C5D0AC0130
:10257000632F61FD70C160FD6EC162FD77C14E5F6A
:10258000534022F119F15523A9F7463398F7483003
:1025900048F00F2DFE2CED2CDC2CCB2CBA2CAA24D1
:1025A0004850A8F7413048F0AA0CBB1CCC1CDD1CDD
:1025B000EE1CFF1C001F4150A9F7702F707E0F7199
:1025C0004EEF53E018D135D1A9F2FBC059C0E8EB6A
:1025D000F9E203C0E8EBF9E20DC05D01FF93EF9370
:1025E00007D2EF91FF913CD0F501FA93EA93C8DE50
:1025F00022960CC25D01FF93EF93FAD1EF91FF9108
:102600002FD0F501FA93EA93A6DE2296FFC1A881A6
:10261000B981661778E06FB78D9195917A9599F0A9
:102620006FBF89076FB7F8CFE881F981AA81BB81B5
:10263000661778E06FB78D9191917A9521F06FBF11
:1026400089076FB7F8CF70E8872797276FBF89078B
:1026500031F06FB7892B12F071E067276FBF0895D3
:1026600088E005900D928A95E1F718970895A08269
:10267000B182C282D382E482F582068317830895F1
:10268000A080B180C280D380E480F580068117816C
:102690000895EC81FD81EBCFE881F981E8CF88E0F6
:1026A00091919D938A95E1F71897389708958681BF
:1026B0009781332797FB37F988949F7721F48823F4
:1026C00011F4326008952FEE28172FE7290740F400
:1026D0002FE02823089411F43160089534600895A0
:1026E000807F9695879596958795969587959695EB
:1026F0008795989488940895A080B180C280D380F3
:10270000E480F58006810F70006122270895108112
:102710003181428153816481758186818F708061AE
:102720000895883050F02A2DAB2CBC2CCD2CDE2CFB
:10273000EF2CF02E00278850F4CF0895689401C044
:10274000E894882369F00595F794E794D794C794A3
:10275000B794A794279516F44F5F5F4F8A95F1CFF2
:102760000895220FAA1CBB1CCC1CDD1CEE1CFF1CF8
:10277000001F089501D025C0203848F011F4A0FEB4
:1027800006C0089412D005FF089581E0D7CF0895C0
:102790002095A094B094C094D094E094F0940095C7
:1027A0000F9200240894201D0F9050F40F920024E3
:1027B000A01CB01CC01CD01CE01CF01C001D0F9005
:1027C00008955523B2F0352F342B99F03FEF43177E
:1027D00037E0530778F4440F551F440F551F440F3B
:1027E000551F440F551F0F7E042B152F67FB17F93C
:1027F000089531C037C087E03F2D303230E0030705
:1028000078F40F2DFE2CED2CDC2CCB2CBA2CA22E28
:102810002227485050408A9579F7442755271BC0F6
:1028200088E004FD05C09DDF415050408A95C9F7FE
:1028300008950F9200240A280B280C280D280E2832
:102840000F28002A00200F900895EA81FB81A881BB
:10285000B9810F010895AA24BB2465017501850182
:1028600098940895F8DF00EF1FE708958FEFA82EE2
:10287000B82EF3DF1F7708951ADF632FAC01FD0137
:1028800016DF732F00C0372F362B3F7709F40895DA
:1028900032FDECCF262F2727372F60FB32F961FB63
:1028A00033F93F70E0ECF9E2002311F427FD3C9688
:1028B000030FE00F0027F01F849187FDD7CF86FD1F
:1028C000D1DF85FDC8DF84FD0AD083FD0AD082FDFB
:1028D0000AD081FD0BD080FD0BD098940895F001B3
:1028E000CFCEFD01CDCE67FB17F9089577FBFCCF66
:1028F00027FBFACFCD90DD90ED90FD90AA24BB246C
:102900000027112722276627FF2012F406D06068CF
:1029100043E254E070DF55DFAACEC094D094E09437
:10292000F09481E0C80E8827D81EE81EF81E08958E
:10293000BEDE31FD19C032FD17C030FD2AC08E5FEA
:10294000934092F0992329F5803238F4D5DE8195B1
:102950008B5DE7DEE894F4DE0CC0CC24C094DC2C64
:10296000EC2CFC2CF69412C0CC24DD24EE24FF24A5
:1029700010C080E8B81650F031F4BA28B22AB81660
:1029800011F4C0FC03C0CDDFF7FCE7CF37FF01C077
:10299000C4DFCD92DD92ED92FD920895B7FE0895C9
:1029A00090E8B91611F4D0FE08959FEFD91AE90AFC
:1029B000F90A09F403950895000000000000F03FB3
:1029C0000008100010101000080820000008100077
:1029D00010801000080820000041200041418000C4
:1029E00020802000002044004180440020208000FE
:1029F00088E00FB6F8945A924A92E42DF52DA42D52
:102A0000B52D480E8827581E0FBE08950FB6F894AE
:102A1000499059900FBE08955A924A92480E591EF5
:102A200008955A924A92480E8827581E0895480ED3
:102A30008827581E08950F921F922F92C801D9011E
:102A4000489F80014A9F90014B9F202C499F100D69
:102A5000211D321D5A9F202C589F100D211D321D03
:102A6000599F200D311D689F200D311D699F300D2C
:102A7000789F300D2F901F900F9008950E94301670
:102A80000D920020D9F70895903029F08C91880F8D
:102A90009A95E9F78C930895903071F00D911D91FE
:102AA0002D913C91000F111F221F331F9A95D1F7D2
:102AB0003C932E931E930E930895903029F08C91A1
:102AC00086959A95E9F78C930895903071F00D9161
:102AD0001D912D913C9136952795179507959A95BF
:102AE000D1F73C932E931E930E93089533D09927DC
:102AF00011278F2D880F80E8F82A802F881F08F46F
:102B00001FEF41F08F57082F07FD04C0003240F03F
:102B10008FEF01C08827982FD82EE82EF82E09C0F5
:102B20008FE1801B082FF694E794D79497950A9528
:102B3000D1F7112351F09095D094E094F09481E076
:102B4000980F8827D81EE81EF81E0F2DFE2CED2C9E
:102B5000D92E0895D190E190F19001910895102F10
:102B600090E8FF0C001F0927990FF7941078652F44
:102B700090E8440F551F5927990F47956078003802
:102B80000895FF0C90E89027110F9795F794092F5F
:102B90000895102FBD2CDE2CEF2CF02E11234AF4BB
:102BA000B094D094E094F0949FEFB91AD90AE90A4E
:102BB000F90A0EE1FF2039F4FE2CED2CDB2CBB24AE
:102BC0000850C2F716C032F00A95BB0CDD1CEE1C93
:102BD000FF1CF9CF0E94CE14D4CFDD92ED92FD926E
:102BE0000C9308959FE7092FF92A9FEFD92EE92E1C
:102BF0000895DD24EE24FF24002711270895AFDF78
:102C0000C1F35038B1F31627005850580894051FE7
:102C100012F418F4E7CF08F0ECCF0BD0FF202AF025
:102C2000BB0CDD1CEE1CFF1CACCF0F5F0BF4DACF2E
:102C3000A8CF9F929924AA24BB24992788E1990CB4
:102C4000AA1CBB1CDD1CEE1CFF1C30F4920EA31E44
:102C5000B41ED91EE91EF91E8A9589F79F90089522
:102C6000C895319600200895FBDF202DF9DF302D27
:102C7000F7DF402DF5DF502D089591E005C092E07B
:102C800003C094E001C098E0EBDF0D929A95E1F764
:102C90000895E80FF91FF1CF2E2E3F2E992781912D
:102CA0008D3209F093958823D1F79A95E22DF32D73
:102CB000112361F0091718F011F0101B01C0191B46
:102CC00028F021F080E28D931A95E9F780818D320A
:102CD00019F48D93319604C0222311F08BE28D9369
:102CE000091738F031F0091B21F080E38D930A9524
:102CF000E9F781918D938823E1F7332351F0EA2F8F
:102D0000FB2F319633958E9182933A95E1F78EE2BF
:102D10008C930895040F151F261F371F0895041B59
:102D2000150B260B370B08950417150726073707D1
:102D30000895000F111F221F331F0895009510954D
:102D4000209530950F5F1F4F2F4F3F4F08950191F2
:102D500010810EC001911191219130810BC0019120
:102D6000108117FF05C03FEF2FEF04C0008111272E
:102D70002227332737FF03C0E1DF8DE28D93CF9306
:102D8000DF93CF92DF92EF92AA24BB24CC24DD24E0
:102D9000EE2440E2CAE0DD2755E093E38881890F05
:102DA00087FD9F7083FD907F891B89935A95A9F7B2
:102DB000C0DFAA1CBB1CCC1CDD1CEE1C4A9551F7C5
:102DC000E894EFE0FF2782910ED0EB30E0F71EF0A1
:102DD00068948A2D0CD088278D93EF90DF90CF9048
:102DE000DF91CF910895982F829501D0892F8F7010
:102DF000805D26F0803309F4089568948D930895DA
:102E000000271127222733271DD08A3328F4803347
:102E100018F005D015D0F9CF0EF490CF0895805357
:102E20008F93402F512F622F732F83DF82DF72DF4A
:102E300080DF8F919927080F191F291F391F0895C7
:102E40008D910895E894FCDF8032E9F38B32D9F359
:102E50008930C9F38D3211F46894F2CF0895882730
:102E60008D93089581918D938823E1F7089594E0DF
:102E700081918D939A95E1F7089509919191992304
:102E800051F08A95D9F7319781918D930A9519F070
:102E90008823D1F70895E3CFE199FECFEEBBFFBBC6
:102EA0003196089591E001C092E07B3751F47FB7ED
:102EB000F894F2DF8D918DBBE29AE19A9A95C9F769
:102EC0007FBF7727089591E001C092E0E5DFE09AA7
:102ED0008DB38D939A95D1F70895FF93881BF9E0F0
:102EE000001FFA9511F4FF910895881F841B18F4B0
:102EF000840F8894F5CF0894F3CF8FEF83959D913D
:102F00009923E1F70895689401C0E894AF93BF93C3
:102F10008D9116F0919103C00E943016902D891763
:102F200018F011F48823A1F7BF91AF910895E894A8
:102F300063F80895689463F80895A998A898A198EB
:102F4000A0980895A09AA19803D0A09801D0A19A22
:102F5000EF93FF93E0E1F0E00E949011FF91EF9179
:102F60000895A09AA19AF4DFA098989BFECFF0DF75
:102F7000A198EECF0894111F01C0110F69F0A09A1B
:102F800018F40000A19802C0A19A00C0E1DFA09847
:102F9000989BFECFDDDFF1CFA09AA198D9DFA09852
:102FA000989BFECFE8949999689462F8D1CF0894E1
:102FB00001C08894331F11E0A09AA198C9DFA0989E
:102FC000989BFECFC5DF889499990894111FA0F7AC
:102FD000A09A379510F4A19801C0A19AB9DFA098E2
:102FE000989BFECFB5DF08950000000000000000B0
:102FF000000000000000B0410000000000DB8A413A
:103000000000001023459B4100000010EE389B415A
:1030100000000090083F9B41000000000000594064
:103020004260653B49463B00494600003B00464143
:0E30300000005A5A50413B005A5A50410000CD
:00000001FF
